:100000000C945C000C946E000C946E000C946E00CA
:100010000C946E000C946E000C946E000C946E00A8
:100020000C946E000C946E000C946E000C946E0098
:100030000C946E000C946E000C946E000C946E0088
:100040000C940F010C946E000C946E000C946E00D6
:100050000C946E000C946E000C946E000C946E0068
:100060000C946E000C946E00000000002400270029
:100070002A0000000000250028002B0004040404CE
:100080000404040402020202020203030303030342
:10009000010204081020408001020408102001021F
:1000A00004081020000000080002010000030407FB
:1000B000000000000000000011241FBECFEFD8E0B8
:1000C000DEBFCDBF21E0A0E0B1E001C01D92A930AC
:1000D000B207E1F70E9459010C9493230C9400009D
:1000E000E6EAF0E02491E2E9F0E09491EEE7F0E056
:1000F000E491EE23C9F0222339F0233001F1A8F472
:10010000213019F1223029F1F0E0EE0FFF1FEE58F7
:10011000FF4FA591B4912FB7F894EC91811126C0AF
:1001200090959E239C932FBF08952730A9F02830E7
:10013000C9F0243049F7209180002F7D03C0209121
:1001400080002F7720938000DFCF24B52F7724BD48
:10015000DBCF24B52F7DFBCF2091B0002F772093EC
:10016000B000D2CF2091B0002F7DF9CF9E2BDACFF7
:100170003FB7F8948091050190910601A091070185
:10018000B091080126B5A89B05C02F3F19F0019634
:10019000A11DB11D3FBFBA2FA92F982F8827BC01E1
:1001A000CD01620F711D811D911D42E0660F771F09
:1001B000881F991F4A95D1F708958F929F92AF9209
:1001C000BF92CF92DF92EF92FF924B015C010E94AF
:1001D000B8006B017C010E94B8006C197D098E0982
:1001E0009F09683E734081059105A8F321E0821ABA
:1001F0009108A108B10888EEC80E83E0D81EE11C62
:10020000F11C81149104A104B10429F7FF90EF902F
:10021000DF90CF90BF90AF909F908F9008951F92E6
:100220000F920FB60F9211242F933F938F939F93AA
:10023000AF93BF938091010190910201A0910301BE
:10024000B09104013091000123E0230F2D3758F5C0
:100250000196A11DB11D209300018093010190938F
:100260000201A0930301B0930401809105019091D4
:100270000601A0910701B09108010196A11DB11DD1
:100280008093050190930601A0930701B0930801A4
:10029000BF91AF919F918F913F912F910F900FBE82
:1002A0000F901F90189526E8230F0296A11DB11DEF
:1002B000D2CF789484B5826084BD84B5816084BDDA
:1002C00085B5826085BD85B5816085BD80916E00F4
:1002D000816080936E001092810080918100826025
:1002E0008093810080918100816080938100809162
:1002F00080008160809380008091B1008460809351
:10030000B1008091B00081608093B00080917A004C
:10031000846080937A0080917A00826080937A0072
:1003200080917A00816080937A0080917A00806861
:1003300080937A001092C100E2E9F0E02491EEE7A8
:10034000F0E08491882399F090E0880F991FFC01D8
:10035000E859FF4FA591B491FC01EE58FF4F8591EC
:1003600094918FB7F894EC91E22BEC938FBFC0E09F
:10037000D0E081E00E94700068EC70E080E090E0E6
:100380000E94DD0080E00E94700068EC70E080E078
:1003900090E00E94DD0081E00E94700068EC70E057
:1003A00080E090E00E94DD0080E00E94700068EC38
:1003B00070E080E090E00E94DD0081E00E9470002B
:1003C00068EC70E080E090E00E94DD0080E00E9438
:1003D000700068EC70E080E090E00E94DD0081E059
:1003E0000E94700068EC70E080E090E00E94DD0008
:1003F00080E00E94700068EC70E080E090E00E9475
:10040000DD0081E00E94700068E572E080E090E02D
:100410000E94DD0080E00E94700068EC70E080E0E7
:1004200090E00E94DD0060E971E080E090E00E94D1
:10043000DD0081E00E94700068E572E080E090E0FD
:100440000E94DD0080E00E94700068EC70E080E0B7
:1004500090E00E94DD0081E00E94700068E572E09B
:1004600080E090E00E94DD0080E00E94700068EC77
:1004700070E080E090E00E94DD0081E00E9470006A
:1004800068E572E080E090E00E94DD0080E00E947C
:10049000700068EC70E080E090E00E94DD0081E098
:1004A0000E94700068E572E080E090E00E94DD004C
:1004B00080E00E94700068EC70E080E090E00E94B4
:1004C000DD0081E00E94700068EC70E080E090E068
:1004D0000E94DD0080E00E94700068EC70E080E027
:1004E00090E00E94DD0060E971E080E090E00E9411
:1004F000DD0081E00E94700068E572E080E090E03D
:100500000E94DD0080E00E94700068EC70E080E0F6
:1005100090E00E94DD0081E00E94700068EC70E0D5
:1005200080E090E00E94DD0080E00E94700068ECB6
:1005300070E080E090E00E94DD0081E00E947000A9
:1005400068EC70E080E090E00E94DD0080E00E94B6
:10055000700068EC70E080E090E00E94DD0081E0D7
:100560000E94700068EC70E080E090E00E94DD0086
:1005700080E00E94700068EC70E080E090E00E94F3
:10058000DD0081E00E94700068EC70E080E090E0A7
:100590000E94DD0080E00E94700068EC70E080E066
:1005A00090E00E94DD0060E971E080E090E00E9450
:1005B000DD0081E00E94700068E572E080E090E07C
:1005C0000E94DD0080E00E94700068EC70E080E036
:1005D00090E00E94DD0081E00E94700068EC70E015
:1005E00080E090E00E94DD0080E00E94700068ECF6
:1005F00070E080E090E00E94DD0081E00E947000E9
:1006000068EC70E080E090E00E94DD0080E00E94F5
:10061000700068EC70E080E090E00E94DD0081E016
:100620000E94700068EC70E080E090E00E94DD00C5
:1006300080E00E94700068EC70E080E090E00E9432
:10064000DD0081E00E94700068EC70E080E090E0E6
:100650000E94DD0080E00E94700068EC70E080E0A5
:1006600090E00E94DD0060E971E080E090E00E948F
:10067000DD0081E00E94700068EC70E080E090E0B6
:100680000E94DD0080E00E94700068EC70E080E075
:1006900090E00E94DD0081E00E94700068EC70E054
:1006A00080E090E00E94DD0080E00E94700068EC35
:1006B00070E080E090E00E94DD0081E00E94700028
:1006C00068E572E080E090E00E94DD0080E00E943A
:1006D000700068EC70E080E090E00E94DD0081E056
:1006E0000E94700068E572E080E090E00E94DD000A
:1006F00080E00E94700068EC70E080E090E00E9472
:10070000DD0081E00E94700068E572E080E090E02A
:100710000E94DD0080E00E94700068EC70E080E0E4
:1007200090E00E94DD0060E971E080E090E00E94CE
:10073000DD0081E00E94700068E572E080E090E0FA
:100740000E94DD0080E00E94700068EC70E080E0B4
:1007500090E00E94DD0081E00E94700068EC70E093
:1007600080E090E00E94DD0080E00E94700068EC74
:1007700070E080E090E00E94DD0081E00E94700067
:1007800068EC70E080E090E00E94DD0080E00E9474
:10079000700068EC70E080E090E00E94DD0060E9AD
:1007A00071E080E090E00E94DD0081E00E94700036
:1007B00068E572E080E090E00E94DD0080E00E9449
:1007C000700068EC70E080E090E00E94DD0081E065
:1007D0000E94700068E572E080E090E00E94DD0019
:1007E00080E00E94700068EC70E080E090E00E9481
:1007F000DD0081E00E94700068EC70E080E090E035
:100800000E94DD0080E00E94700068EC70E080E0F3
:1008100090E00E94DD0081E00E94700068EC70E0D2
:1008200080E090E00E94DD0080E00E94700068ECB3
:1008300070E080E090E00E94DD0081E00E947000A6
:1008400068EC70E080E090E00E94DD0080E00E94B3
:10085000700068EC70E080E090E00E94DD0060E9EC
:1008600071E080E090E00E94DD0081E00E94700075
:1008700068E572E080E090E00E94DD0080E00E9488
:10088000700068EC70E080E090E00E94DD0081E0A4
:100890000E94700068E572E080E090E00E94DD0058
:1008A00080E00E94700068EC70E080E090E00E94C0
:1008B000DD0081E00E94700068E572E080E090E079
:1008C0000E94DD0080E00E94700068EC70E080E033
:1008D00090E00E94DD0081E00E94700068E572E017
:1008E00080E090E00E94DD0080E00E94700068ECF3
:1008F00070E080E090E00E94DD0081E00E947000E6
:1009000068EC70E080E090E00E94DD0080E00E94F2
:10091000700068EC70E080E090E00E94DD0060E92B
:1009200071E080E090E00E94DD0081E00E947000B4
:1009300068E572E080E090E00E94DD0080E00E94C7
:10094000700068EC70E080E090E00E94DD0081E0E3
:100950000E94700068EC70E080E090E00E94DD0092
:1009600080E00E94700068EC70E080E090E00E94FF
:10097000DD0081E00E94700068EC70E080E090E0B3
:100980000E94DD0080E00E94700068EC70E080E072
:1009900090E00E94DD0081E00E94700068EC70E051
:1009A00080E090E00E94DD0080E00E94700068EC32
:1009B00070E080E090E00E94DD0081E00E94700025
:1009C00068EC70E080E090E00E94DD0080E00E9432
:1009D000700068EC70E080E090E00E94DD0060E96B
:1009E00071E080E090E00E94DD0081E00E947000F4
:1009F00068EC70E080E090E00E94DD0080E00E9402
:100A0000700068EC70E080E090E00E94DD0081E022
:100A10000E94700068EC70E080E090E00E94DD00D1
:100A200080E00E94700068EC70E080E090E00E943E
:100A3000DD0081E00E94700068E572E080E090E0F7
:100A40000E94DD0080E00E94700068EC70E080E0B1
:100A500090E00E94DD0081E00E94700068EC70E090
:100A600080E090E00E94DD0080E00E94700068EC71
:100A700070E080E090E00E94DD0060E971E080E0DD
:100A800090E00E94DD0081E00E94700068E572E065
:100A900080E090E00E94DD0080E00E94700068EC41
:100AA00070E080E090E00E94DD0081E00E94700034
:100AB00068E572E080E090E00E94DD0080E00E9446
:100AC000700068EC70E080E090E00E94DD0081E062
:100AD0000E94700068EC70E080E090E00E94DD0011
:100AE00080E00E94700068EC70E080E090E00E947E
:100AF000DD0081E00E94700068EC70E080E090E032
:100B00000E94DD0080E00E94700068EC70E080E0F0
:100B100090E00E94DD0081E00E94700068EC70E0CF
:100B200080E090E00E94DD0080E00E94700068ECB0
:100B300070E080E090E00E94DD0060E971E080E01C
:100B400090E00E94DD0081E00E94700068EC70E09F
:100B500080E090E00E94DD0080E00E94700068EC80
:100B600070E080E090E00E94DD0081E00E94700073
:100B700068EC70E080E090E00E94DD0080E00E9480
:100B8000700068EC70E080E090E00E94DD0081E0A1
:100B90000E94700068EC70E080E090E00E94DD0050
:100BA00080E00E94700068EC70E080E090E00E94BD
:100BB000DD0081E00E94700068EC70E080E090E071
:100BC0000E94DD0080E00E94700068EC70E080E030
:100BD00090E00E94DD0081E00E94700068EC70E00F
:100BE00080E090E00E94DD0080E00E94700068ECF0
:100BF00070E080E090E00E94DD0060E971E080E05C
:100C000090E00E94DD0081E00E94700068EC70E0DE
:100C100080E090E00E94DD0080E00E94700068ECBF
:100C200070E080E090E00E94DD0081E00E947000B2
:100C300068EC70E080E090E00E94DD0080E00E94BF
:100C4000700068EC70E080E090E00E94DD0081E0E0
:100C50000E94700068E572E080E090E00E94DD0094
:100C600080E00E94700068EC70E080E090E00E94FC
:100C7000DD0081E00E94700068E572E080E090E0B5
:100C80000E94DD0080E00E94700068EC70E080E06F
:100C900090E00E94DD0081E00E94700068E572E053
:100CA00080E090E00E94DD0080E00E94700068EC2F
:100CB00070E080E090E00E94DD0060E971E080E09B
:100CC00090E00E94DD0081E00E94700068E572E023
:100CD00080E090E00E94DD0080E00E94700068ECFF
:100CE00070E080E090E00E94DD0081E00E947000F2
:100CF00068EC70E080E090E00E94DD0080E00E94FF
:100D0000700068EC70E080E090E00E94DD0081E01F
:100D10000E94700068EC70E080E090E00E94DD00CE
:100D200080E00E94700068EC70E080E090E00E943B
:100D3000DD0060E971E080E090E00E94DD0081E08C
:100D40000E94700068E572E080E090E00E94DD00A3
:100D500080E00E94700068EC70E080E090E00E940B
:100D6000DD0081E00E94700068EC70E080E090E0BF
:100D70000E94DD0080E00E94700068EC70E080E07E
:100D800090E00E94DD0081E00E94700068EC70E05D
:100D900080E090E00E94DD0080E00E94700068EC3E
:100DA00070E080E090E00E94DD0081E00E94700031
:100DB00068EC70E080E090E00E94DD0080E00E943E
:100DC000700068EC70E080E090E00E94DD0081E05F
:100DD0000E94700068EC70E080E090E00E94DD000E
:100DE00080E00E94700068EC70E080E090E00E947B
:100DF000DD0060E971E080E090E00E94DD0081E0CC
:100E00000E94700068EC70E080E090E00E94DD00DD
:100E100080E00E94700068EC70E080E090E00E944A
:100E2000DD0081E00E94700068EC70E080E090E0FE
:100E30000E94DD0080E00E94700068EC70E080E0BD
:100E400090E00E94DD0081E00E94700068EC70E09C
:100E500080E090E00E94DD0080E00E94700068EC7D
:100E600070E080E090E00E94DD0081E00E94700070
:100E700068EC70E080E090E00E94DD0080E00E947D
:100E8000700068EC70E080E090E00E94DD0081E09E
:100E90000E94700068E572E080E090E00E94DD0052
:100EA00080E00E94700068EC70E080E090E00E94BA
:100EB000DD0060E971E080E090E00E94DD0081E00B
:100EC0000E94700068E572E080E090E00E94DD0022
:100ED00080E00E94700068EC70E080E090E00E948A
:100EE000DD0081E00E94700068EC70E080E090E03E
:100EF0000E94DD0080E00E94700068EC70E080E0FD
:100F000090E00E94DD0081E00E94700068EC70E0DB
:100F100080E090E00E94DD0080E00E94700068ECBC
:100F200070E080E090E00E94DD0081E00E947000AF
:100F300068EC70E080E090E00E94DD0080E00E94BC
:100F4000700068EC70E080E090E00E94DD0081E0DD
:100F50000E94700068EC70E080E090E00E94DD008C
:100F600080E00E94700068EC70E080E090E00E94F9
:100F7000DD0060E971E080E090E00E94DD0081E04A
:100F80000E94700068E572E080E090E00E94DD0061
:100F900080E00E94700068EC70E080E090E00E94C9
:100FA000DD0081E00E94700068E572E080E090E082
:100FB0000E94DD0080E00E94700068EC70E080E03C
:100FC00090E00E94DD0081E00E94700068E572E020
:100FD00080E090E00E94DD0080E00E94700068ECFC
:100FE00070E080E090E00E94DD0081E00E947000EF
:100FF00068E572E080E090E00E94DD0080E00E9401
:10100000700068EC70E080E090E00E94DD0081E01C
:101010000E94700068EC70E080E090E00E94DD00CB
:1010200080E00E94700068EC70E080E090E00E9438
:10103000DD0060E971E080E090E00E94DD0081E089
:101040000E94700068E572E080E090E00E94DD00A0
:1010500080E00E94700068EC70E080E090E00E9408
:10106000DD0081E00E94700068EC70E080E090E0BC
:101070000E94DD0080E00E94700068EC70E080E07B
:1010800090E00E94DD0081E00E94700068EC70E05A
:1010900080E090E00E94DD0080E00E94700068EC3B
:1010A00070E080E090E00E94DD0081E00E9470002E
:1010B00068EC70E080E090E00E94DD0080E00E943B
:1010C000700068EC70E080E090E00E94DD0081E05C
:1010D0000E94700068EC70E080E090E00E94DD000B
:1010E00080E00E94700068EC70E080E090E00E9478
:1010F000DD0060E971E080E090E00E94DD0081E0C9
:101100000E94700068EC70E080E090E00E94DD00DA
:1011100080E00E94700068EC70E080E090E00E9447
:10112000DD0081E00E94700068EC70E080E090E0FB
:101130000E94DD0080E00E94700068EC70E080E0BA
:1011400090E00E94DD0081E00E94700068EC70E099
:1011500080E090E00E94DD0080E00E94700068EC7A
:1011600070E080E090E00E94DD0081E00E9470006D
:1011700068EC70E080E090E00E94DD0080E00E947A
:10118000700068EC70E080E090E00E94DD0081E09B
:101190000E94700068E572E080E090E00E94DD004F
:1011A00080E00E94700068EC70E080E090E00E94B7
:1011B000DD0060E971E080E090E00E94DD0081E008
:1011C0000E94700068EC70E080E090E00E94DD001A
:1011D00080E00E94700068EC70E080E090E00E9487
:1011E000DD0081E00E94700068EC70E080E090E03B
:1011F0000E94DD0080E00E94700068EC70E080E0FA
:1012000090E00E94DD0081E00E94700068E572E0DD
:1012100080E090E00E94DD0080E00E94700068ECB9
:1012200070E080E090E00E94DD0081E00E947000AC
:1012300068E572E080E090E00E94DD0080E00E94BE
:10124000700068EC70E080E090E00E94DD0081E0DA
:101250000E94700068E572E080E090E00E94DD008E
:1012600080E00E94700068EC70E080E090E00E94F6
:10127000DD0060E971E080E090E00E94DD0081E047
:101280000E94700068E572E080E090E00E94DD005E
:1012900080E00E94700068EC70E080E090E00E94C6
:1012A000DD0081E00E94700068EC70E080E090E07A
:1012B0000E94DD0080E00E94700068EC70E080E039
:1012C00090E00E94DD0081E00E94700068EC70E018
:1012D00080E090E00E94DD0080E00E94700068ECF9
:1012E00070E080E090E00E94DD0060E971E080E065
:1012F00090E00E94DD0081E00E94700068E572E0ED
:1013000080E090E00E94DD0080E00E94700068ECC8
:1013100070E080E090E00E94DD0081E00E947000BB
:1013200068EC70E080E090E00E94DD0080E00E94C8
:10133000700068EC70E080E090E00E94DD0081E0E9
:101340000E94700068EC70E080E090E00E94DD0098
:1013500080E00E94700068EC70E080E090E00E9405
:10136000DD0081E00E94700068EC70E080E090E0B9
:101370000E94DD0080E00E94700068EC70E080E078
:1013800090E00E94DD0081E00E94700068EC70E057
:1013900080E090E00E94DD0080E00E94700068EC38
:1013A00070E080E090E00E94DD0060E971E080E0A4
:1013B00090E00E94DD0081E00E94700068EC70E027
:1013C00080E090E00E94DD0080E00E94700068EC08
:1013D00070E080E090E00E94DD0060E971E080E074
:1013E00090E00E94DD0081E00E94700068E572E0FC
:1013F00080E090E00E94DD0080E00E94700068ECD8
:1014000070E080E090E00E94DD0081E00E947000CA
:1014100068EC70E080E090E00E94DD0080E00E94D7
:10142000700068EC70E080E090E00E94DD0081E0F8
:101430000E94700068EC70E080E090E00E94DD00A7
:1014400080E00E94700068EC70E080E090E00E9414
:10145000DD0081E00E94700068EC70E080E090E0C8
:101460000E94DD0080E00E94700068EC70E080E087
:1014700090E00E94DD0081E00E94700068EC70E066
:1014800080E090E00E94DD0080E00E94700068EC47
:1014900070E080E090E00E94DD0060E971E080E0B3
:1014A00090E00E94DD0081E00E94700068EC70E036
:1014B00080E090E00E94DD0080E00E94700068EC17
:1014C00070E080E090E00E94DD0081E00E9470000A
:1014D00068EC70E080E090E00E94DD0080E00E9417
:1014E000700068EC70E080E090E00E94DD0081E038
:1014F0000E94700068E572E080E090E00E94DD00EC
:1015000080E00E94700068EC70E080E090E00E9453
:10151000DD0081E00E94700068EC70E080E090E007
:101520000E94DD0080E00E94700068EC70E080E0C6
:1015300090E00E94DD0060E971E080E090E00E94B0
:10154000DD0081E00E94700068E572E080E090E0DC
:101550000E94DD0080E00E94700068EC70E080E096
:1015600090E00E94DD0081E00E94700068E572E07A
:1015700080E090E00E94DD0080E00E94700068EC56
:1015800070E080E090E00E94DD0081E00E94700049
:1015900068EC70E080E090E00E94DD0080E00E9456
:1015A000700068EC70E080E090E00E94DD0081E077
:1015B0000E94700068EC70E080E090E00E94DD0026
:1015C00080E00E94700068EC70E080E090E00E9493
:1015D000DD0081E00E94700068EC70E080E090E047
:1015E0000E94DD0080E00E94700068EC70E080E006
:1015F00090E00E94DD0060E971E080E090E00E94F0
:10160000DD0081E00E94700068EC70E080E090E016
:101610000E94DD0080E00E94700068EC70E080E0D5
:1016200090E00E94DD0081E00E94700068EC70E0B4
:1016300080E090E00E94DD0080E00E94700068EC95
:1016400070E080E090E00E94DD0081E00E94700088
:1016500068EC70E080E090E00E94DD0080E00E9495
:10166000700068EC70E080E090E00E94DD0081E0B6
:101670000E94700068EC70E080E090E00E94DD0065
:1016800080E00E94700068EC70E080E090E00E94D2
:10169000DD0081E00E94700068E572E080E090E08B
:1016A0000E94DD0080E00E94700068EC70E080E045
:1016B00090E00E94DD0060E971E080E090E00E942F
:1016C000DD0081E00E94700068EC70E080E090E056
:1016D0000E94DD0080E00E94700068EC70E080E015
:1016E00090E00E94DD0081E00E94700068EC70E0F4
:1016F00080E090E00E94DD0080E00E94700068ECD5
:1017000070E080E090E00E94DD0081E00E947000C7
:1017100068E572E080E090E00E94DD0080E00E94D9
:10172000700068EC70E080E090E00E94DD0081E0F5
:101730000E94700068E572E080E090E00E94DD00A9
:1017400080E00E94700068EC70E080E090E00E9411
:10175000DD0081E00E94700068E572E080E090E0CA
:101760000E94DD0080E00E94700068EC70E080E084
:1017700090E00E94DD0060E971E080E090E00E946E
:10178000DD0081E00E94700068E572E080E090E09A
:101790000E94DD0080E00E94700068EC70E080E054
:1017A00090E00E94DD0081E00E94700068EC70E033
:1017B00080E090E00E94DD0080E00E94700068EC14
:1017C00070E080E090E00E94DD0081E00E94700007
:1017D00068EC70E080E090E00E94DD0080E00E9414
:1017E000700068EC70E080E090E00E94DD0060E94D
:1017F00071E080E090E00E94DD0081E00E947000D6
:1018000068E572E080E090E00E94DD0080E00E94E8
:10181000700068EC70E080E090E00E94DD0081E004
:101820000E94700068E572E080E090E00E94DD00B8
:1018300080E00E94700068EC70E080E090E00E9420
:10184000DD0081E00E94700068EC70E080E090E0D4
:101850000E94DD0080E00E94700068EC70E080E093
:1018600090E00E94DD0081E00E94700068EC70E072
:1018700080E090E00E94DD0080E00E94700068EC53
:1018800070E080E090E00E94DD0081E00E94700046
:1018900068EC70E080E090E00E94DD0080E00E9453
:1018A000700068EC70E080E090E00E94DD0060E98C
:1018B00071E080E090E00E94DD0081E00E94700015
:1018C00068EC70E080E090E00E94DD0080E00E9423
:1018D000700068EC70E080E090E00E94DD0081E044
:1018E0000E94700068EC70E080E090E00E94DD00F3
:1018F00080E00E94700068EC70E080E090E00E9460
:10190000DD0081E00E94700068EC70E080E090E013
:101910000E94DD0080E00E94700068EC70E080E0D2
:1019200090E00E94DD0081E00E94700068E572E0B6
:1019300080E090E00E94DD0080E00E94700068EC92
:1019400070E080E090E00E94DD0081E00E94700085
:1019500068E572E080E090E00E94DD0080E00E9497
:10196000700068EC70E080E090E00E94DD0060E9CB
:1019700071E080E090E00E94DD0081E00E94700054
:1019800068E572E080E090E00E94DD0080E00E9467
:10199000700068EC70E080E090E00E94DD0081E083
:1019A0000E94700068EC70E080E090E00E94DD0032
:1019B00080E00E94700068EC70E080E090E00E949F
:1019C000DD0081E00E94700068EC70E080E090E053
:1019D0000E94DD0080E00E94700068EC70E080E012
:1019E00090E00E94DD0081E00E94700068EC70E0F1
:1019F00080E090E00E94DD0080E00E94700068ECD2
:101A000070E080E090E00E94DD0081E00E947000C4
:101A100068EC70E080E090E00E94DD0080E00E94D1
:101A2000700068EC70E080E090E00E94DD0060E90A
:101A300071E080E090E00E94DD0081E00E94700093
:101A400068EC70E080E090E00E94DD0080E00E94A1
:101A5000700068EC70E080E090E00E94DD0081E0C2
:101A60000E94700068EC70E080E090E00E94DD0071
:101A700080E00E94700068EC70E080E090E00E94DE
:101A8000DD0081E00E94700068EC70E080E090E092
:101A90000E94DD0080E00E94700068EC70E080E051
:101AA00090E00E94DD0081E00E94700068E572E035
:101AB00080E090E00E94DD0080E00E94700068EC11
:101AC00070E080E090E00E94DD0081E00E94700004
:101AD00068E572E080E090E00E94DD0080E00E9416
:101AE000700068EC70E080E090E00E94DD0060E94A
:101AF00071E080E090E00E94DD0081E00E947000D3
:101B000068E572E080E090E00E94DD0080E00E94E5
:101B1000700068EC70E080E090E00E94DD0081E001
:101B20000E94700068E572E080E090E00E94DD00B5
:101B300080E00E94700068EC70E080E090E00E941D
:101B4000DD0081E00E94700068EC70E080E090E0D1
:101B50000E94DD0080E00E94700068EC70E080E090
:101B600090E00E94DD0081E00E94700068EC70E06F
:101B700080E090E00E94DD0080E00E94700068EC50
:101B800070E080E090E00E94DD0081E00E94700043
:101B900068EC70E080E090E00E94DD0080E00E9450
:101BA000700068EC70E080E090E00E94DD0060E989
:101BB00071E080E090E00E94DD0081E00E94700012
:101BC00068EC70E080E090E00E94DD0080E00E9420
:101BD000700068EC70E080E090E00E94DD0081E041
:101BE0000E94700068EC70E080E090E00E94DD00F0
:101BF00080E00E94700068EC70E080E090E00E945D
:101C0000DD0081E00E94700068E572E080E090E015
:101C10000E94DD0080E00E94700068EC70E080E0CF
:101C200090E00E94DD0081E00E94700068E572E0B3
:101C300080E090E00E94DD0080E00E94700068EC8F
:101C400070E080E090E00E94DD0081E00E94700082
:101C500068E572E080E090E00E94DD0080E00E9494
:101C6000700068EC70E080E090E00E94DD0060E9C8
:101C700071E080E090E00E94DD0081E00E94700051
:101C800068E572E080E090E00E94DD0080E00E9464
:101C9000700068EC70E080E090E00E94DD0081E080
:101CA0000E94700068EC70E080E090E00E94DD002F
:101CB00080E00E94700068EC70E080E090E00E949C
:101CC000DD0081E00E94700068EC70E080E090E050
:101CD0000E94DD0080E00E94700068EC70E080E00F
:101CE00090E00E94DD0081E00E94700068EC70E0EE
:101CF00080E090E00E94DD0080E00E94700068ECCF
:101D000070E080E090E00E94DD0081E00E947000C1
:101D100068EC70E080E090E00E94DD0080E00E94CE
:101D2000700068EC70E080E090E00E94DD0060E907
:101D300071E080E090E00E94DD0081E00E94700090
:101D400068E572E080E090E00E94DD0080E00E94A3
:101D5000700068EC70E080E090E00E94DD0081E0BF
:101D60000E94700068E572E080E090E00E94DD0073
:101D700080E00E94700068EC70E080E090E00E94DB
:101D8000DD0081E00E94700068E572E080E090E094
:101D90000E94DD0080E00E94700068EC70E080E04E
:101DA00090E00E94DD0081E00E94700068E572E032
:101DB00080E090E00E94DD0080E00E94700068EC0E
:101DC00070E080E090E00E94DD0081E00E94700001
:101DD00068EC70E080E090E00E94DD0080E00E940E
:101DE000700068EC70E080E090E00E94DD0060E947
:101DF00071E080E090E00E94DD0081E00E947000D0
:101E000068E572E080E090E00E94DD0080E00E94E2
:101E1000700068EC70E080E090E00E94DD0081E0FE
:101E20000E94700068E572E080E090E00E94DD00B2
:101E300080E00E94700068EC70E080E090E00E941A
:101E4000DD0081E00E94700068EC70E080E090E0CE
:101E50000E94DD0080E00E94700068EC70E080E08D
:101E600090E00E94DD0081E00E94700068EC70E06C
:101E700080E090E00E94DD0080E00E94700068EC4D
:101E800070E080E090E00E94DD0081E00E94700040
:101E900068EC70E080E090E00E94DD0080E00E944D
:101EA000700068EC70E080E090E00E94DD0060E986
:101EB00071E080E090E00E94DD0081E00E9470000F
:101EC00068E572E080E090E00E94DD0080E00E9422
:101ED000700068EC70E080E090E00E94DD0081E03E
:101EE0000E94700068E572E080E090E00E94DD00F2
:101EF00080E00E94700068EC70E080E090E00E945A
:101F0000DD0081E00E94700068E572E080E090E012
:101F10000E94DD0080E00E94700068EC70E080E0CC
:101F200090E00E94DD0081E00E94700068E572E0B0
:101F300080E090E00E94DD0080E00E94700068EC8C
:101F400070E080E090E00E94DD0081E00E9470007F
:101F500068E572E080E090E00E94DD0080E00E9491
:101F6000700068EC70E080E090E00E94DD0060E9C5
:101F700071E080E090E00E94DD0081E00E9470004E
:101F800068E572E080E090E00E94DD0080E00E9461
:101F9000700068EC70E080E090E00E94DD0081E07D
:101FA0000E94700068E572E080E090E00E94DD0031
:101FB00080E00E94700068EC70E080E090E00E9499
:101FC000DD0081E00E94700068EC70E080E090E04D
:101FD0000E94DD0080E00E94700068EC70E080E00C
:101FE00090E00E94DD0081E00E94700068EC70E0EB
:101FF00080E090E00E94DD0080E00E94700068ECCC
:1020000070E080E090E00E94DD0081E00E947000BE
:1020100068EC70E080E090E00E94DD0080E00E94CB
:10202000700068EC70E080E090E00E94DD0060E904
:1020300071E080E090E00E94DD0081E00E9470008D
:1020400068EC70E080E090E00E94DD0080E00E949B
:10205000700068EC70E080E090E00E94DD0081E0BC
:102060000E94700068EC70E080E090E00E94DD006B
:1020700080E00E94700068EC70E080E090E00E94D8
:10208000DD0081E00E94700068EC70E080E090E08C
:102090000E94DD0080E00E94700068EC70E080E04B
:1020A00090E00E94DD0081E00E94700068EC70E02A
:1020B00080E090E00E94DD0080E00E94700068EC0B
:1020C00070E080E090E00E94DD0081E00E947000FE
:1020D00068E572E080E090E00E94DD0080E00E9410
:1020E000700068EC70E080E090E00E94DD0060E944
:1020F00071E080E090E00E94DD0081E00E947000CD
:1021000068EC70E080E090E00E94DD0080E00E94DA
:10211000700068EC70E080E090E00E94DD0081E0FB
:102120000E94700068EC70E080E090E00E94DD00AA
:1021300080E00E94700068EC70E080E090E00E9417
:10214000DD0081E00E94700068E572E080E090E0D0
:102150000E94DD0080E00E94700068EC70E080E08A
:1021600090E00E94DD0081E00E94700068E572E06E
:1021700080E090E00E94DD0080E00E94700068EC4A
:1021800070E080E090E00E94DD0081E00E9470003D
:1021900068E572E080E090E00E94DD0080E00E944F
:1021A000700068EC70E080E090E00E94DD0060E983
:1021B00071E080E090E00E94DD0081E00E9470000C
:1021C00068E572E080E090E00E94DD0080E00E941F
:1021D000700068EC70E080E090E00E94DD0081E03B
:1021E0000E94700068EC70E080E090E00E94DD00EA
:1021F00080E00E94700068EC70E080E090E00E9457
:10220000DD0081E00E94700068EC70E080E090E00A
:102210000E94DD0080E00E94700068EC70E080E0C9
:1022200090E00E94DD0060E971E080E090E00E94B3
:10223000DD0081E00E94700068E572E080E090E0DF
:102240000E94DD0080E00E94700068EC70E080E099
:1022500090E00E94DD0081E00E94700068E572E07D
:1022600080E090E00E94DD0080E00E94700068EC59
:1022700070E080E090E00E94DD0081E00E9470004C
:1022800068EC70E080E090E00E94DD0080E00E9459
:10229000700068EC70E080E090E00E94DD0081E07A
:1022A0000E94700068EC70E080E090E00E94DD0029
:1022B00080E00E94700068EC70E080E090E00E9496
:1022C000DD0081E00E94700068EC70E080E090E04A
:1022D0000E94DD0080E00E94700068EC70E080E009
:1022E00090E00E94DD0060E971E080E090E00E94F3
:1022F000DD0081E00E94700068E572E080E090E01F
:102300000E94DD0080E00E94700068EC70E080E0D8
:1023100090E00E94DD0081E00E94700068E572E0BC
:1023200080E090E00E94DD0080E00E94700068EC98
:1023300070E080E090E00E94DD0081E00E9470008B
:1023400068E572E080E090E00E94DD0080E00E949D
:10235000700068EC70E080E090E00E94DD0081E0B9
:102360000E94700068E572E080E090E00E94DD006D
:1023700080E00E94700068EC70E080E090E00E94D5
:10238000DD0081E00E94700068EC70E080E090E089
:102390000E94DD0080E00E94700068EC70E080E048
:1023A00090E00E94DD0060E971E080E090E00E9432
:1023B000DD0081E00E94700068E572E080E090E05E
:1023C0000E94DD0080E00E94700068EC70E080E018
:1023D00090E00E94DD0081E00E94700068EC70E0F7
:1023E00080E090E00E94DD0080E00E94700068ECD8
:1023F00070E080E090E00E94DD0081E00E947000CB
:1024000068EC70E080E090E00E94DD0080E00E94D7
:10241000700068EC70E080E090E00E94DD0081E0F8
:102420000E94700068EC70E080E090E00E94DD00A7
:1024300080E00E94700068EC70E080E090E00E9414
:10244000DD0081E00E94700068EC70E080E090E0C8
:102450000E94DD0080E00E94700068EC70E080E087
:1024600090E00E94DD0060E971E080E090E00E9471
:10247000DD0081E00E94700068EC70E080E090E098
:102480000E94DD0080E00E94700068EC70E080E057
:1024900090E00E94DD0081E00E94700068EC70E036
:1024A00080E090E00E94DD0080E00E94700068EC17
:1024B00070E080E090E00E94DD0081E00E9470000A
:1024C00068E572E080E090E00E94DD0080E00E941C
:1024D000700068EC70E080E090E00E94DD0081E038
:1024E0000E94700068EC70E080E090E00E94DD00E7
:1024F00080E00E94700068EC70E080E090E00E9454
:10250000DD0060E971E080E090E00E94DD0081E0A4
:102510000E94700068E572E080E090E00E94DD00BB
:1025200080E00E94700068EC70E080E090E00E9423
:10253000DD0081E00E94700068E572E080E090E0DC
:102540000E94DD0080E00E94700068EC70E080E096
:1025500090E00E94DD0081E00E94700068EC70E075
:1025600080E090E00E94DD0080E00E94700068EC56
:1025700070E080E090E00E94DD0081E00E94700049
:1025800068EC70E080E090E00E94DD0080E00E9456
:10259000700068EC70E080E090E00E94DD0081E077
:1025A0000E94700068EC70E080E090E00E94DD0026
:1025B00080E00E94700068EC70E080E090E00E9493
:1025C000DD0060E971E080E090E00E94DD0081E0E4
:1025D0000E94700068EC70E080E090E00E94DD00F6
:1025E00080E00E94700068EC70E080E090E00E9463
:1025F000DD0081E00E94700068EC70E080E090E017
:102600000E94DD0080E00E94700068EC70E080E0D5
:1026100090E00E94DD0081E00E94700068EC70E0B4
:1026200080E090E00E94DD0080E00E94700068EC95
:1026300070E080E090E00E94DD0081E00E94700088
:1026400068EC70E080E090E00E94DD0080E00E9495
:10265000700068EC70E080E090E00E94DD0081E0B6
:102660000E94700068EC70E080E090E00E94DD0065
:1026700080E00E94700068EC70E080E090E00E94D2
:10268000DD0060E971E080E090E00E94DD0081E023
:102690000E94700068EC70E080E090E00E94DD0035
:1026A00080E00E94700068EC70E080E090E00E94A2
:1026B000DD0081E00E94700068EC70E080E090E056
:1026C0000E94DD0080E00E94700068EC70E080E015
:1026D00090E00E94DD0081E00E94700068E572E0F9
:1026E00080E090E00E94DD0080E00E94700068ECD5
:1026F00070E080E090E00E94DD0081E00E947000C8
:1027000068E572E080E090E00E94DD0080E00E94D9
:10271000700068EC70E080E090E00E94DD0081E0F5
:102720000E94700068E572E080E090E00E94DD00A9
:1027300080E00E94700068EC70E080E090E00E9411
:10274000DD0060E971E080E090E00E94DD0081E062
:102750000E94700068E572E080E090E00E94DD0079
:1027600080E00E94700068EC70E080E090E00E94E1
:10277000DD0081E00E94700068EC70E080E090E095
:102780000E94DD0080E00E94700068EC70E080E054
:1027900090E00E94DD0081E00E94700068EC70E033
:1027A00080E090E00E94DD0080E00E94700068EC14
:1027B00070E080E090E00E94DD0060E971E080E080
:1027C00090E00E94DD0081E00E94700068E572E008
:1027D00080E090E00E94DD0080E00E94700068ECE4
:1027E00070E080E090E00E94DD0081E00E947000D7
:1027F00068EC70E080E090E00E94DD0080E00E94E4
:10280000700068EC70E080E090E00E94DD0081E004
:102810000E94700068EC70E080E090E00E94DD00B3
:1028200080E00E94700068EC70E080E090E00E9420
:10283000DD0081E00E94700068EC70E080E090E0D4
:102840000E94DD0080E00E94700068EC70E080E093
:1028500090E00E94DD0081E00E94700068EC70E072
:1028600080E090E00E94DD0080E00E94700068EC53
:1028700070E080E090E00E94DD0060E971E080E0BF
:1028800090E00E94DD0081E00E94700068E572E047
:1028900080E090E00E94DD0080E00E94700068EC23
:1028A00070E080E090E00E94DD0081E00E94700016
:1028B00068EC70E080E090E00E94DD0080E00E9423
:1028C000700068EC70E080E090E00E94DD0081E044
:1028D0000E94700068EC70E080E090E00E94DD00F3
:1028E00080E00E94700068EC70E080E090E00E9460
:1028F000DD0060E971E080E090E00E94DD0081E0B1
:102900000E94700068E572E080E090E00E94DD00C7
:1029100080E00E94700068EC70E080E090E00E942F
:10292000DD0081E00E94700068E572E080E090E0E8
:102930000E94DD0080E00E94700068EC70E080E0A2
:1029400090E00E94DD0081E00E94700068EC70E081
:1029500080E090E00E94DD0080E00E94700068EC62
:1029600070E080E090E00E94DD0081E00E94700055
:1029700068EC70E080E090E00E94DD0080E00E9462
:10298000700068EC70E080E090E00E94DD0081E083
:102990000E94700068EC70E080E090E00E94DD0032
:1029A00080E00E94700068EC70E080E090E00E949F
:1029B000DD0060E971E080E090E00E94DD0081E0F0
:1029C0000E94700068EC70E080E090E00E94DD0002
:1029D00080E00E94700068EC70E080E090E00E946F
:1029E000DD0081E00E94700068EC70E080E090E023
:1029F0000E94DD0080E00E94700068EC70E080E0E2
:102A000090E00E94DD0081E00E94700068EC70E0C0
:102A100080E090E00E94DD0080E00E94700068ECA1
:102A200070E080E090E00E94DD0081E00E94700094
:102A300068EC70E080E090E00E94DD0080E00E94A1
:102A4000700068EC70E080E090E00E94DD0081E0C2
:102A50000E94700068EC70E080E090E00E94DD0071
:102A600080E00E94700068EC70E080E090E00E94DE
:102A7000DD0060E971E080E090E00E94DD0081E02F
:102A80000E94700068E572E080E090E00E94DD0046
:102A900080E00E94700068EC70E080E090E00E94AE
:102AA000DD0081E00E94700068E572E080E090E067
:102AB0000E94DD0080E00E94700068EC70E080E021
:102AC00090E00E94DD0081E00E94700068EC70E000
:102AD00080E090E00E94DD0080E00E94700068ECE1
:102AE00070E080E090E00E94DD0081E00E947000D4
:102AF00068EC70E080E090E00E94DD0080E00E94E1
:102B0000700068EC70E080E090E00E94DD0081E001
:102B10000E94700068EC70E080E090E00E94DD00B0
:102B200080E00E94700068EC70E080E090E00E941D
:102B3000DD0060E971E080E090E00E94DD0081E06E
:102B40000E94700068EC70E080E090E00E94DD0080
:102B500080E00E94700068EC70E080E090E00E94ED
:102B6000DD0081E00E94700068EC70E080E090E0A1
:102B70000E94DD0080E00E94700068EC70E080E060
:102B800090E00E94DD0081E00E94700068EC70E03F
:102B900080E090E00E94DD0080E00E94700068EC20
:102BA00070E080E090E00E94DD0081E00E94700013
:102BB00068E572E080E090E00E94DD0080E00E9425
:102BC000700068EC70E080E090E00E94DD0081E041
:102BD0000E94700068E572E080E090E00E94DD00F5
:102BE00080E00E94700068EC70E080E090E00E945D
:102BF000DD0060E971E080E090E00E94DD0081E0AE
:102C00000E94700068E572E080E090E00E94DD00C4
:102C100080E00E94700068EC70E080E090E00E942C
:102C2000DD0081E00E94700068E572E080E090E0E5
:102C30000E94DD0080E00E94700068EC70E080E09F
:102C400090E00E94DD0081E00E94700068EC70E07E
:102C500080E090E00E94DD0080E00E94700068EC5F
:102C600070E080E090E00E94DD0081E00E94700052
:102C700068EC70E080E090E00E94DD0080E00E945F
:102C8000700068EC70E080E090E00E94DD0081E080
:102C90000E94700068EC70E080E090E00E94DD002F
:102CA00080E00E94700068EC70E080E090E00E949C
:102CB000DD0060E971E080E090E00E94DD0081E0ED
:102CC0000E94700068EC70E080E090E00E94DD00FF
:102CD00080E00E94700068EC70E080E090E00E946C
:102CE000DD0081E00E94700068EC70E080E090E020
:102CF0000E94DD0080E00E94700068EC70E080E0DF
:102D000090E00E94DD0081E00E94700068EC70E0BD
:102D100080E090E00E94DD0080E00E94700068EC9E
:102D200070E080E090E00E94DD0081E00E94700091
:102D300068EC70E080E090E00E94DD0080E00E949E
:102D4000700068EC70E080E090E00E94DD0081E0BF
:102D50000E94700068E572E080E090E00E94DD0073
:102D600080E00E94700068EC70E080E090E00E94DB
:102D7000DD0060E971E080E090E00E94DD0081E02C
:102D80000E94700068EC70E080E090E00E94DD003E
:102D900080E00E94700068EC70E080E090E00E94AB
:102DA000DD0081E00E94700068EC70E080E090E05F
:102DB0000E94DD0080E00E94700068EC70E080E01E
:102DC00090E00E94DD0081E00E94700068E572E002
:102DD00080E090E00E94DD0080E00E94700068ECDE
:102DE00070E080E090E00E94DD0081E00E947000D1
:102DF00068E572E080E090E00E94DD0080E00E94E3
:102E0000700068EC70E080E090E00E94DD0081E0FE
:102E10000E94700068E572E080E090E00E94DD00B2
:102E200080E00E94700068EC70E080E090E00E941A
:102E3000DD0060E971E080E090E00E94DD0081E06B
:102E40000E94700068E572E080E090E00E94DD0082
:102E500080E00E94700068EC70E080E090E00E94EA
:102E6000DD0081E00E94700068EC70E080E090E09E
:102E70000E94DD0080E00E94700068EC70E080E05D
:102E800090E00E94DD0081E00E94700068EC70E03C
:102E900080E090E00E94DD0080E00E94700068EC1D
:102EA00070E080E090E00E94DD0060E971E080E089
:102EB00090E00E94DD0081E00E94700068E572E011
:102EC00080E090E00E94DD0080E00E94700068ECED
:102ED00070E080E090E00E94DD0081E00E947000E0
:102EE00068EC70E080E090E00E94DD0080E00E94ED
:102EF000700068EC70E080E090E00E94DD0081E00E
:102F00000E94700068EC70E080E090E00E94DD00BC
:102F100080E00E94700068EC70E080E090E00E9429
:102F2000DD0081E00E94700068EC70E080E090E0DD
:102F30000E94DD0080E00E94700068EC70E080E09C
:102F400090E00E94DD0081E00E94700068EC70E07B
:102F500080E090E00E94DD0080E00E94700068EC5C
:102F600070E080E090E00E94DD0060E971E080E0C8
:102F700090E00E94DD0081E00E94700068EC70E04B
:102F800080E090E00E94DD0080E00E94700068EC2C
:102F900070E080E090E00E94DD0081E00E9470001F
:102FA00068EC70E080E090E00E94DD0080E00E942C
:102FB000700068EC70E080E090E00E94DD0081E04D
:102FC0000E94700068E572E080E090E00E94DD0001
:102FD00080E00E94700068EC70E080E090E00E9469
:102FE000DD0081E00E94700068E572E080E090E022
:102FF0000E94DD0080E00E94700068EC70E080E0DC
:1030000090E00E94DD0081E00E94700068E572E0BF
:1030100080E090E00E94DD0080E00E94700068EC9B
:1030200070E080E090E00E94DD0060E971E080E007
:1030300090E00E94DD0081E00E94700068E572E08F
:1030400080E090E00E94DD0080E00E94700068EC6B
:1030500070E080E090E00E94DD0081E00E9470005E
:1030600068EC70E080E090E00E94DD0080E00E946B
:10307000700068EC70E080E090E00E94DD0081E08C
:103080000E94700068EC70E080E090E00E94DD003B
:1030900080E00E94700068EC70E080E090E00E94A8
:1030A000DD0081E00E94700068EC70E080E090E05C
:1030B0000E94DD0080E00E94700068EC70E080E01B
:1030C00090E00E94DD0081E00E94700068EC70E0FA
:1030D00080E090E00E94DD0080E00E94700068ECDB
:1030E00070E080E090E00E94DD0060E971E080E047
:1030F00090E00E94DD0081E00E94700068EC70E0CA
:1031000080E090E00E94DD0080E00E94700068ECAA
:1031100070E080E090E00E94DD0081E00E9470009D
:1031200068EC70E080E090E00E94DD0080E00E94AA
:10313000700068EC70E080E090E00E94DD0081E0CB
:103140000E94700068EC70E080E090E00E94DD007A
:1031500080E00E94700068EC70E080E090E00E94E7
:10316000DD0081E00E94700068EC70E080E090E09B
:103170000E94DD0080E00E94700068EC70E080E05A
:1031800090E00E94DD0081E00E94700068EC70E039
:1031900080E090E00E94DD0080E00E94700068EC1A
:1031A00070E080E090E00E94DD0060E971E080E086
:1031B00090E00E94DD0081E00E94700068EC70E009
:1031C00080E090E00E94DD0080E00E94700068ECEA
:1031D00070E080E090E00E94DD0081E00E947000DD
:1031E00068EC70E080E090E00E94DD0080E00E94EA
:1031F000700068EC70E080E090E00E94DD0081E00B
:103200000E94700068E572E080E090E00E94DD00BE
:1032100080E00E94700068EC70E080E090E00E9426
:10322000DD0081E00E94700068E572E080E090E0DF
:103230000E94DD0080E00E94700068EC70E080E099
:1032400090E00E94DD0081E00E94700068E572E07D
:1032500080E090E00E94DD0080E00E94700068EC59
:1032600070E080E090E00E94DD0060E971E080E0C5
:1032700090E00E94DD0081E00E94700068E572E04D
:1032800080E090E00E94DD0080E00E94700068EC29
:1032900070E080E090E00E94DD0081E00E9470001C
:1032A00068EC70E080E090E00E94DD0080E00E9429
:1032B000700068EC70E080E090E00E94DD0081E04A
:1032C0000E94700068EC70E080E090E00E94DD00F9
:1032D00080E00E94700068EC70E080E090E00E9466
:1032E000DD0060E971E080E090E00E94DD0081E0B7
:1032F0000E94700068EC70E080E090E00E94DD00C9
:1033000080E00E94700068EC70E080E090E00E9435
:10331000DD0081E00E94700068EC70E080E090E0E9
:103320000E94DD0080E00E94700068EC70E080E0A8
:1033300090E00E94DD0081E00E94700068EC70E087
:1033400080E090E00E94DD0080E00E94700068EC68
:1033500070E080E090E00E94DD0081E00E9470005B
:1033600068E572E080E090E00E94DD0080E00E946D
:10337000700068EC70E080E090E00E94DD0081E089
:103380000E94700068E572E080E090E00E94DD003D
:1033900080E00E94700068EC70E080E090E00E94A5
:1033A000DD0060E971E080E090E00E94DD0081E0F6
:1033B0000E94700068EC70E080E090E00E94DD0008
:1033C00080E00E94700068EC70E080E090E00E9475
:1033D000DD0081E00E94700068E572E080E090E02E
:1033E0000E94DD0080E00E94700068EC70E080E0E8
:1033F00090E00E94DD0081E00E94700068E572E0CC
:1034000080E090E00E94DD0080E00E94700068ECA7
:1034100070E080E090E00E94DD0081E00E9470009A
:1034200068E572E080E090E00E94DD0080E00E94AC
:10343000700068EC70E080E090E00E94DD0081E0C8
:103440000E94700068E572E080E090E00E94DD007C
:1034500080E00E94700068EC70E080E090E00E94E4
:10346000DD0060E971E080E090E00E94DD0081E035
:103470000E94700068EC70E080E090E00E94DD0047
:1034800080E00E94700068EC70E080E090E00E94B4
:10349000DD0081E00E94700068EC70E080E090E068
:1034A0000E94DD0080E00E94700068EC70E080E027
:1034B00090E00E94DD0081E00E94700068EC70E006
:1034C00080E090E00E94DD0080E00E94700068ECE7
:1034D00070E080E090E00E94DD0081E00E947000DA
:1034E00068E572E080E090E00E94DD0080E00E94EC
:1034F000700068EC70E080E090E00E94DD0081E008
:103500000E94700068E572E080E090E00E94DD00BB
:1035100080E00E94700068EC70E080E090E00E9423
:10352000DD0060E971E080E090E00E94DD0081E074
:103530000E94700068E572E080E090E00E94DD008B
:1035400080E00E94700068EC70E080E090E00E94F3
:10355000DD0081E00E94700068E572E080E090E0AC
:103560000E94DD0080E00E94700068EC70E080E066
:1035700090E00E94DD0081E00E94700068E572E04A
:1035800080E090E00E94DD0080E00E94700068EC26
:1035900070E080E090E00E94DD0081E00E94700019
:1035A00068E572E080E090E00E94DD0080E00E942B
:1035B000700068EC70E080E090E00E94DD0081E047
:1035C0000E94700068E572E080E090E00E94DD00FB
:1035D00080E00E94700068EC70E080E090E00E9463
:1035E000DD0060E971E080E090E00E94DD0081E0B4
:1035F0000E94700068EC70E080E090E00E94DD00C6
:1036000080E00E94700068EC70E080E090E00E9432
:10361000DD0081E00E94700068EC70E080E090E0E6
:103620000E94DD0080E00E94700068EC70E080E0A5
:1036300090E00E94DD0081E00E94700068EC70E084
:1036400080E090E00E94DD0080E00E94700068EC65
:1036500070E080E090E00E94DD0081E00E94700058
:1036600068E572E080E090E00E94DD0080E00E946A
:10367000700068EC70E080E090E00E94DD0081E086
:103680000E94700068E572E080E090E00E94DD003A
:1036900080E00E94700068EC70E080E090E00E94A2
:1036A000DD0060E971E080E090E00E94DD0081E0F3
:1036B0000E94700068E572E080E090E00E94DD000A
:1036C00080E00E94700068EC70E080E090E00E9472
:1036D000DD0081E00E94700068E572E080E090E02B
:1036E0000E94DD0080E00E94700068EC70E080E0E5
:1036F00090E00E94DD0081E00E94700068E572E0C9
:1037000080E090E00E94DD0080E00E94700068ECA4
:1037100070E080E090E00E94DD0081E00E94700097
:1037200068E572E080E090E00E94DD0080E00E94A9
:10373000700068EC70E080E090E00E94DD0081E0C5
:103740000E94700068E572E080E090E00E94DD0079
:1037500080E00E94700068EC70E080E090E00E94E1
:10376000DD0060E971E080E090E00E94DD0081E032
:103770000E94700068EC70E080E090E00E94DD0044
:1037800080E00E94700068EC70E080E090E00E94B1
:10379000DD0081E00E94700068EC70E080E090E065
:1037A0000E94DD0080E00E94700068EC70E080E024
:1037B00090E00E94DD0081E00E94700068E572E008
:1037C00080E090E00E94DD0080E00E94700068ECE4
:1037D00070E080E090E00E94DD0081E00E947000D7
:1037E00068E572E080E090E00E94DD0080E00E94E9
:1037F000700068EC70E080E090E00E94DD0081E005
:103800000E94700068E572E080E090E00E94DD00B8
:1038100080E00E94700068EC70E080E090E00E9420
:10382000DD0060E971E080E090E00E94DD0081E071
:103830000E94700068E572E080E090E00E94DD0088
:1038400080E00E94700068EC70E080E090E00E94F0
:10385000DD0081E00E94700068EC70E080E090E0A4
:103860000E94DD0080E00E94700068EC70E080E063
:1038700090E00E94DD0081E00E94700068EC70E042
:1038800080E090E00E94DD0080E00E94700068EC23
:1038900070E080E090E00E94DD0060E971E080E08F
:1038A00090E00E94DD0081E00E94700068E572E017
:1038B00080E090E00E94DD0080E00E94700068ECF3
:1038C00070E080E090E00E94DD0081E00E947000E6
:1038D00068E572E080E090E00E94DD0080E00E94F8
:1038E000700068EC70E080E090E00E94DD0081E014
:1038F0000E94700068EC70E080E090E00E94DD00C3
:1039000080E00E94700068EC70E080E090E00E942F
:10391000DD0081E00E94700068EC70E080E090E0E3
:103920000E94DD0080E00E94700068EC70E080E0A2
:1039300090E00E94DD0081E00E94700068EC70E081
:1039400080E090E00E94DD0080E00E94700068EC62
:1039500070E080E090E00E94DD0060E971E080E0CE
:1039600090E00E94DD0081E00E94700068E572E056
:1039700080E090E00E94DD0080E00E94700068EC32
:1039800070E080E090E00E94DD0081E00E94700025
:1039900068E572E080E090E00E94DD0080E00E9437
:1039A000700068EC70E080E090E00E94DD0081E053
:1039B0000E94700068E572E080E090E00E94DD0007
:1039C00080E00E94700068EC70E080E090E00E946F
:1039D000DD0081E00E94700068E572E080E090E028
:1039E0000E94DD0080E00E94700068EC70E080E0E2
:1039F00090E00E94DD0081E00E94700068EC70E0C1
:103A000080E090E00E94DD0080E00E94700068ECA1
:103A100070E080E090E00E94DD0060E971E080E00D
:103A200090E00E94DD0081E00E94700068E572E095
:103A300080E090E00E94DD0080E00E94700068EC71
:103A400070E080E090E00E94DD0081E00E94700064
:103A500068EC70E080E090E00E94DD0080E00E9471
:103A6000700068EC70E080E090E00E94DD0081E092
:103A70000E94700068EC70E080E090E00E94DD0041
:103A800080E00E94700068EC70E080E090E00E94AE
:103A9000DD0081E00E94700068EC70E080E090E062
:103AA0000E94DD0080E00E94700068EC70E080E021
:103AB00090E00E94DD0081E00E94700068EC70E000
:103AC00080E090E00E94DD0080E00E94700068ECE1
:103AD00070E080E090E00E94DD0060E971E080E04D
:103AE00090E00E94DD0081E00E94700068EC70E0D0
:103AF00080E090E00E94DD0080E00E94700068ECB1
:103B000070E080E090E00E94DD0081E00E947000A3
:103B100068EC70E080E090E00E94DD0080E00E94B0
:103B2000700068EC70E080E090E00E94DD0081E0D1
:103B30000E94700068EC70E080E090E00E94DD0080
:103B400080E00E94700068EC70E080E090E00E94ED
:103B5000DD0081E00E94700068EC70E080E090E0A1
:103B60000E94DD0080E00E94700068EC70E080E060
:103B700090E00E94DD0081E00E94700068EC70E03F
:103B800080E090E00E94DD0080E00E94700068EC20
:103B900070E080E090E00E94DD0060E971E080E08C
:103BA00090E00E94DD0081E00E94700068E572E014
:103BB00080E090E00E94DD0080E00E94700068ECF0
:103BC00070E080E090E00E94DD0081E00E947000E3
:103BD00068EC70E080E090E00E94DD0080E00E94F0
:103BE000700068EC70E080E090E00E94DD0081E011
:103BF0000E94700068EC70E080E090E00E94DD00C0
:103C000080E00E94700068EC70E080E090E00E942C
:103C1000DD0081E00E94700068EC70E080E090E0E0
:103C20000E94DD0080E00E94700068EC70E080E09F
:103C300090E00E94DD0081E00E94700068EC70E07E
:103C400080E090E00E94DD0080E00E94700068EC5F
:103C500070E080E090E00E94DD0060E971E080E0CB
:103C600090E00E94DD0081E00E94700068EC70E04E
:103C700080E090E00E94DD0080E00E94700068EC2F
:103C800070E080E090E00E94DD0081E00E94700022
:103C900068E572E080E090E00E94DD0080E00E9434
:103CA000700068EC70E080E090E00E94DD0081E050
:103CB0000E94700068E572E080E090E00E94DD0004
:103CC00080E00E94700068EC70E080E090E00E946C
:103CD000DD0081E00E94700068E572E080E090E025
:103CE0000E94DD0080E00E94700068EC70E080E0DF
:103CF00090E00E94DD0081E00E94700068E572E0C3
:103D000080E090E00E94DD0080E00E94700068EC9E
:103D100070E080E090E00E94DD0060E971E080E00A
:103D200090E00E94DD0081E00E94700068E572E092
:103D300080E090E00E94DD0080E00E94700068EC6E
:103D400070E080E090E00E94DD0081E00E94700061
:103D500068E572E080E090E00E94DD0080E00E9473
:103D6000700068EC70E080E090E00E94DD0081E08F
:103D70000E94700068EC70E080E090E00E94DD003E
:103D800080E00E94700068EC70E080E090E00E94AB
:103D9000DD0081E00E94700068EC70E080E090E05F
:103DA0000E94DD0080E00E94700068EC70E080E01E
:103DB00090E00E94DD0081E00E94700068EC70E0FD
:103DC00080E090E00E94DD0080E00E94700068ECDE
:103DD00070E080E090E00E94DD0060E971E080E04A
:103DE00090E00E94DD0081E00E94700068EC70E0CD
:103DF00080E090E00E94DD0080E00E94700068ECAE
:103E000070E080E090E00E94DD0081E00E947000A0
:103E100068EC70E080E090E00E94DD0080E00E94AD
:103E2000700068EC70E080E090E00E94DD0081E0CE
:103E30000E94700068E572E080E090E00E94DD0082
:103E400080E00E94700068EC70E080E090E00E94EA
:103E5000DD0081E00E94700068E572E080E090E0A3
:103E60000E94DD0080E00E94700068EC70E080E05D
:103E700090E00E94DD0081E00E94700068E572E041
:103E800080E090E00E94DD0080E00E94700068EC1D
:103E900070E080E090E00E94DD0060E971E080E089
:103EA00090E00E94DD0081E00E94700068E572E011
:103EB00080E090E00E94DD0080E00E94700068ECED
:103EC00070E080E090E00E94DD0081E00E947000E0
:103ED00068E572E080E090E00E94DD0080E00E94F2
:103EE000700068EC70E080E090E00E94DD0081E00E
:103EF0000E94700068EC70E080E090E00E94DD00BD
:103F000080E00E94700068EC70E080E090E00E9429
:103F1000DD0081E00E94700068EC70E080E090E0DD
:103F20000E94DD0080E00E94700068EC70E080E09C
:103F300090E00E94DD0081E00E94700068EC70E07B
:103F400080E090E00E94DD0080E00E94700068EC5C
:103F500070E080E090E00E94DD0060E971E080E0C8
:103F600090E00E94DD0081E00E94700068EC70E04B
:103F700080E090E00E94DD0080E00E94700068EC2C
:103F800070E080E090E00E94DD0081E00E9470001F
:103F900068EC70E080E090E00E94DD0080E00E942C
:103FA000700068EC70E080E090E00E94DD0081E04D
:103FB0000E94700068EC70E080E090E00E94DD00FC
:103FC00080E00E94700068EC70E080E090E00E9469
:103FD000DD0081E00E94700068E572E080E090E022
:103FE0000E94DD0080E00E94700068EC70E080E0DC
:103FF00090E00E94DD0081E00E94700068E572E0C0
:1040000080E090E00E94DD0080E00E94700068EC9B
:1040100070E080E090E00E94DD0060E971E080E007
:1040200090E00E94DD0081E00E94700068EC70E08A
:1040300080E090E00E94DD0080E00E94700068EC6B
:1040400070E080E090E00E94DD0081E00E9470005E
:1040500068EC70E080E090E00E94DD0080E00E946B
:10406000700068EC70E080E090E00E94DD0081E08C
:104070000E94700068E572E080E090E00E94DD0040
:1040800080E00E94700068EC70E080E090E00E94A8
:10409000DD0081E00E94700068E572E080E090E061
:1040A0000E94DD0080E00E94700068EC70E080E01B
:1040B00090E00E94DD0081E00E94700068E572E0FF
:1040C00080E090E00E94DD0080E00E94700068ECDB
:1040D00070E080E090E00E94DD0060E971E080E047
:1040E00090E00E94DD0081E00E94700068E572E0CF
:1040F00080E090E00E94DD0080E00E94700068ECAB
:1041000070E080E090E00E94DD0081E00E9470009D
:1041100068EC70E080E090E00E94DD0080E00E94AA
:10412000700068EC70E080E090E00E94DD0081E0CB
:104130000E94700068EC70E080E090E00E94DD007A
:1041400080E00E94700068EC70E080E090E00E94E7
:10415000DD0060E971E080E090E00E94DD0081E038
:104160000E94700068E572E080E090E00E94DD004F
:1041700080E00E94700068EC70E080E090E00E94B7
:10418000DD0081E00E94700068EC70E080E090E06B
:104190000E94DD0080E00E94700068EC70E080E02A
:1041A00090E00E94DD0081E00E94700068EC70E009
:1041B00080E090E00E94DD0080E00E94700068ECEA
:1041C00070E080E090E00E94DD0081E00E947000DD
:1041D00068EC70E080E090E00E94DD0080E00E94EA
:1041E000700068EC70E080E090E00E94DD0081E00B
:1041F0000E94700068EC70E080E090E00E94DD00BA
:1042000080E00E94700068EC70E080E090E00E9426
:10421000DD0060E971E080E090E00E94DD0081E077
:104220000E94700068EC70E080E090E00E94DD0089
:1042300080E00E94700068EC70E080E090E00E94F6
:10424000DD0081E00E94700068EC70E080E090E0AA
:104250000E94DD0080E00E94700068EC70E080E069
:1042600090E00E94DD0081E00E94700068E572E04D
:1042700080E090E00E94DD0080E00E94700068EC29
:1042800070E080E090E00E94DD0081E00E9470001C
:1042900068EC70E080E090E00E94DD0080E00E9429
:1042A000700068EC70E080E090E00E94DD0060E962
:1042B00071E080E090E00E94DD0081E00E947000EB
:1042C00068E572E080E090E00E94DD0080E00E94FE
:1042D000700068EC70E080E090E00E94DD0081E01A
:1042E0000E94700068EC70E080E090E00E94DD00C9
:1042F00080E00E94700068EC70E080E090E00E9436
:10430000DD0081E00E94700068EC70E080E090E0E9
:104310000E94DD0080E00E94700068EC70E080E0A8
:1043200090E00E94DD0081E00E94700068EC70E087
:1043300080E090E00E94DD0080E00E94700068EC68
:1043400070E080E090E00E94DD0081E00E9470005B
:1043500068EC70E080E090E00E94DD0080E00E9468
:10436000700068EC70E080E090E00E94DD0060E9A1
:1043700071E080E090E00E94DD0081E00E9470002A
:1043800068E572E080E090E00E94DD0080E00E943D
:10439000700068EC70E080E090E00E94DD0081E059
:1043A0000E94700068EC70E080E090E00E94DD0008
:1043B00080E00E94700068EC70E080E090E00E9475
:1043C000DD0081E00E94700068E572E080E090E02E
:1043D0000E94DD0080E00E94700068EC70E080E0E8
:1043E00090E00E94DD0081E00E94700068EC70E0C7
:1043F00080E090E00E94DD0080E00E94700068ECA8
:1044000070E080E090E00E94DD0060E971E080E013
:1044100090E00E94DD0081E00E94700068E572E09B
:1044200080E090E00E94DD0080E00E94700068EC77
:1044300070E080E090E00E94DD0081E00E9470006A
:1044400068EC70E080E090E00E94DD0080E00E9477
:10445000700068EC70E080E090E00E94DD0081E098
:104460000E94700068EC70E080E090E00E94DD0047
:1044700080E00E94700068EC70E080E090E00E94B4
:10448000DD0081E00E94700068EC70E080E090E068
:104490000E94DD0080E00E94700068EC70E080E027
:1044A00090E00E94DD0081E00E94700068EC70E006
:1044B00080E090E00E94DD0080E00E94700068ECE7
:1044C00070E080E090E00E94DD0060E971E080E053
:1044D00090E00E94DD0081E00E94700068EC70E0D6
:1044E00080E090E00E94DD0080E00E94700068ECB7
:1044F00070E080E090E00E94DD0081E00E947000AA
:1045000068EC70E080E090E00E94DD0080E00E94B6
:10451000700068EC70E080E090E00E94DD0081E0D7
:104520000E94700068EC70E080E090E00E94DD0086
:1045300080E00E94700068EC70E080E090E00E94F3
:10454000DD0081E00E94700068EC70E080E090E0A7
:104550000E94DD0080E00E94700068EC70E080E066
:1045600090E00E94DD0081E00E94700068E572E04A
:1045700080E090E00E94DD0080E00E94700068EC26
:1045800070E080E090E00E94DD0060E971E080E092
:1045900090E00E94DD0081E00E94700068EC70E015
:1045A00080E090E00E94DD0080E00E94700068ECF6
:1045B00070E080E090E00E94DD0081E00E947000E9
:1045C00068EC70E080E090E00E94DD0080E00E94F6
:1045D000700068EC70E080E090E00E94DD0081E017
:1045E0000E94700068E572E080E090E00E94DD00CB
:1045F00080E00E94700068EC70E080E090E00E9433
:10460000DD0081E00E94700068E572E080E090E0EB
:104610000E94DD0080E00E94700068EC70E080E0A5
:1046200090E00E94DD0081E00E94700068E572E089
:1046300080E090E00E94DD0080E00E94700068EC65
:1046400070E080E090E00E94DD0060E971E080E0D1
:1046500090E00E94DD0081E00E94700068EC70E054
:1046600080E090E00E94DD0080E00E94700068EC35
:1046700070E080E090E00E94DD0081E00E94700028
:1046800068E572E080E090E00E94DD0080E00E943A
:10469000700068EC70E080E090E00E94DD0081E056
:1046A0000E94700068E572E080E090E00E94DD000A
:1046B00080E00E94700068EC70E080E090E00E9472
:1046C000DD0081E00E94700068E572E080E090E02B
:1046D0000E94DD0080E00E94700068EC70E080E0E5
:1046E00090E00E94DD0081E00E94700068E572E0C9
:1046F00080E090E00E94DD0080E00E94700068ECA5
:1047000070E080E090E00E94DD0060E971E080E010
:1047100090E00E94DD00209711F40C94B9010E94F2
:0A47200000000C94B901F894FFCFDB
:00000001FF
